:107000004FC00000A7C00000A5C00000A3C0000042
:10701000A1C000009FC000009DC000009BC00000F8
:1070200099C0000097C0000095C0000093C0000008
:1070300091C000008FC000008DC000008BC0000018
:1070400089C0000087C0000085C0000083C0000028
:1070500081C000007FC000007DC000007BC0000038
:1070600079C0000077C0000000050000496E76611D
:107070006C696420696D61676500000500004572F8
:10708000726F720000050003466C617368204675DC
:107090006C6C00000500044F70636F64653F000076
:1070A00011241FBECFEFD8E0DEBFCDBF14E0A0E0BB
:1070B000B1E0E4EAF9E702C005900D92AA30B10709
:1070C000D9F714E0AAE0B4E001C01D92A331B107E2
:1070D000E1F701D065C414BE88E10FB6F89480933F
:1070E0006000109260000FBEF4D32FEF84E39CE0A9
:1070F000215080409040E1F700C000008EE284B94A
:107100008CE385B983E08093810081E08DBD8CE1C3
:1071100091E0EED38DE491E0EBD381E591E0E8D30B
:10712000A6D081E691E0E4D381E791E0E1D33ED3BC
:1071300080E891E0DDD356D3882311F00CD0FBCF4B
:1071400081E991E0D5D3E0910A04F0910B0409950F
:1071500080E090E055CF20918400309185008091AF
:107160001104909112042817390770F480910C04CF
:1071700090910D04019690930D0480930C04299B2B
:1071800002C0299801C0299A309312042093110457
:107190000895E0E0F0E085919491019641F081E05E
:1071A00020910C0430910D042431310508F480E065
:1071B000089510920D0410920C04089520E52CBD42
:1071C0002A9820EF2EBD0DB407FEFDCF292F3327BF
:1071D0002EBD0DB407FEFDCF8EBD0DB407FEFDCF55
:1071E0006EBD0DB407FEFDCF2A9A1CBC089520E5A4
:1071F0002CBD2A982FE02EBD0DB407FEFDCF292F00
:1072000033272EBD0DB407FEFDCF8EBD0DB407FE96
:10721000FDCF1EBC0DB407FEFDCF2A9A8EB51CBC57
:1072200008950F931F93CF938C01E1DFC82FC801FE
:107230000196DDDF2C2F30E0322F2227A901482BC9
:10724000CA01CF911F910F9108950F931F93CF9370
:10725000DF93EC018B01672F7727CE01AFDF602F23
:10726000CE010196DF91CF911F910F91A7CF0F9380
:107270001F93CF93DF9380E090E07CD38535A9F412
:1072800081E090E077D38A3A81F482EA91E030D3CA
:10729000C3E0D0E0CE016ED3FE01E250FF4F808309
:1072A0002196C531D105B1F703C08AEB91E020D317
:1072B00000E011E0C0E0D0E0F80161918F01CE0163
:1072C0007DDF2196CC31D105B9F7DF91CF911F91A8
:1072D0000F9108954F925F926F927F928F929F923B
:1072E000AF92BF92CF92DF92EF92FF920F931F93D4
:1072F000CF93DF93CDB7DEB7C051D240DEBFCDBF55
:107300008C0183ED91E0F4D280E192E0F1D289E248
:1073100092E0EED2C8010BD38AE392E0E9D20115E4
:10732000184019F483E492E0E3D288E297E079DF31
:107330004C0181E0881688E0980678F081E592E0BB
:10734000D7D289E992E0D4D2C401F1D28EE492E09E
:10735000CFD2340197E0792201C0340189E992E06B
:10736000C7D2C3019858E3D26301EAEFCE1AE7E827
:10737000DE0AC6013CDF082FC301895F974837DF6B
:1073800010E0102F0027080F111D7801F8E0EF0E14
:10739000F11C8EE492E0ACD282E792E0A9D2C60161
:1073A000C6D28EE492E0A4D283E892E0A1D2580142
:1073B00024E0A21AB108C501BAD28EE492E098D2B4
:1073C000CE0101966C012C01073F8FEF180791F059
:1073D000C30198580CDFF20181932F01FFEF6F1A60
:1073E0007F0A611428E0720611F4612C712C01509F
:1073F0001109EACF85E992E07BD28E0C9F1CC40173
:1074000096D28EE492E074D2B40188E297E01DDF58
:1074100060E481E097E0D2DE81E097E0E8DE811170
:10742000FBCF87EA92E064D286E297E0FADE7FD271
:107430008EE492E05DD286019CE0892E97E0992E41
:1074400026E0722E7C0CF80161918F01C401B6DE3A
:10745000FFEF8F1A9F0A7012F6CF8984912C982C17
:1074600088248A85880E911C0B8510E0102F002738
:107470008C85080F111D84EB92E03AD2C80157D2D7
:107480008EE492E035D285EC92E032D2C4014FD244
:107490008EE492E02DD223E08216910409F453C0C9
:1074A00028F492E08916910491F00AC0E4E08E1667
:1074B000910409F4C1C0F5E08F16910409F4BFC02E
:1074C000C40135D28DEC92E013D281E0BEC081EED2
:1074D00092E00ED260E481E097E070DE60E181E04E
:1074E00097E06CDE62E080E097E068DE61E081E0DA
:1074F00097E064DE6E8170E0609570958D81782BE9
:1075000084E097E0A2DE83E097E071DE823221F032
:1075100060E181E097E052DE83E097E068DE82324E
:1075200009F781EF92E0E4D19E8185E589272D81DD
:1075300090E0922BFCD18EE492E0DAD1109210040C
:1075400010920F0481C01093100400930F04015097
:107550001109102F0027110F82E093E0C9D180910B
:107560000F0490911004E3D18EE492E0C1D1C701E1
:10757000800F911F8130904728F08CE193E0B8D1C3
:1075800083E063C08DE293E0B3D1C801D0D18EE433
:1075900092E0AED1C7018F779927892B21F08FEF29
:1075A000E81AF80AF7CF0115110551F4CE010D962E
:1075B0007DD1811105C088E493E09AD185E045C072
:1075C00020E030E041E053E065E071E12E153F0539
:1075D00050F5F601E20FF31F858590E0982F88277C
:1075E000E4858E2BF8010C0140935700E895112497
:1075F0002E5F3F4FC9018F779927892B89F4EE576A
:10760000F10950935700E89507B600FCFDCF609351
:107610005700E89507B600FCFDCF70935700E8953A
:107620000E5F1F4FD3CFA114F2E0BF0668F489E5C7
:1076300093E05ED184E009C08DE693E002C083E769
:1076400093E056D180E001C082E0C05FDD4FDEBF35
:10765000CDBFDF91CF911F910F91FF90EF90DF9001
:10766000CF90BF90AF909F908F907F906F905F90E2
:107670004F900895CF92DF92EF92FF920F931F9356
:10768000CF93DF93CDB7DEB7C556D109DEBFCDBFEF
:107690008C0184E297E0C5DD985A7C010330110526
:1076A00061F138F401301105F9F00230110571F182
:1076B00006C00430110569F10530110561F04AE09A
:1076C00050E06AE770E7CE0101964BD12AE08E01C7
:1076D0000F5F1F4F4BC042E150E068E670E7CE01FC
:1076E00001963FD122E1F3CF4CE050E063E970E72F
:1076F000CE01019636D12CE0EACF4FE050E064E8AD
:1077000070E7CE0101962DD12FE0E1CF8BE793E01A
:10771000EFD082E993E0ECD080910F0490911004B7
:1077200006D18EE492E0E4D0198284E08A838091CD
:107730000F04909110049B838C8324E0C8CFF80140
:1077400061918F016701FFEFCF1ADF0AC701A6968B
:107750002FAFA69733DDA6962FADA697C11480E66E
:10776000D80619F4C12C88E5D82E7601215038F7B7
:10777000B701785584E297E068DD60E281E097E048
:107780001DDD81E097E033DD8111FBCF8CE993E0D3
:10779000AFD0CB59DF4FDEBFCDBFDF91CF911F916F
:1077A0000F91FF90EF90DF90CF90089565E470E027
:1077B00084E097E04ADD62E080E097E0FFDC61E092
:1077C00081E097E0FBDC83E097E011DD823221F07D
:1077D00060E181E097E0F2DC83E097E008DD82324F
:1077E00029F70895CF9386E297E01BDD009731F1EA
:1077F00071DDC82F90E03EDF81E080930E046FEFD3
:1078000082E090E0BFD0D5DCC430C1F460E181E01B
:1078100097E0D4DC6BEB82E090E0B4D08CEA93E0AC
:1078200067D082E090E0A6D090E081D08EE492E034
:107830005FD085EB93E05CD0C0E035C0AADC882344
:10784000E9F080910E048823C9F060E181E097E0BF
:10785000B5DC85EC93E04CD08DED93E049D01092EF
:107860000E0407B600FCFDCFF999FECFE0E0F0E092
:1078700083E080935700E89599DF14C08ADC882361
:1078800089F0C0910E04C1110DC082E090E072D069
:107890008B3B41F460E181E097E090DC8EEF93E078
:1078A00027D001C0C1E08C2FCF910895FC01319603
:1078B000C596DF0111972C912C3049F42081243991
:1078C00031F43496E817F907A1F781E0089580E0D4
:1078D000089582E28093C00088E08093C10080E137
:1078E00090E09093C5008093C40082E98AB908951E
:1078F000FC019191992339F09093C6008091C000CA
:1079000085FFFCCFF6CF08958093C6008091C0001C
:1079100085FFFCCF08958F708A3008F0895F805D05
:107920008093C6008091C00085FFFCCF0895CF935F
:10793000DF93EC0180E3E8DF88E7E6DFCE01892F03
:10794000992782958F70E7DF8D2FE5DFCE0134E038
:10795000969587953A95E1F7DEDF8C2FDF91CF91F1
:10796000DACFFB01DC0102C005900D92415050407E
:10797000D8F70895F999FECF92BD81BDF89A99275D
:1079800080B50895262FF999FECF1FBA92BD81BD0B
:1079900020BD0FB6F894FA9AF99A0FBE0196089591
:0479A000F894FFCF89
:1079A40080C0A80001FFFFFC000008DCBD25FFC06B
:1079B400A800B40000000007D08055550D0A5446B5
:1079C400545020426F6F746C6F6164657220666FEF
:1079D400722041726475696E6F2045746865726EB9
:1079E40065742C2056657273696F6E2000302E32D8
:1079F400000D0A4E657420696E69742E2E2E0D0AD0
:107A0400004E657420696E697420646F6E650D0A9A
:107A1400005446545020496E69742E2E2E0D0A00CF
:107A24005446545020496E697420646F6E650D0A83
:107A34000053746172742075736572206170700DE7
:107A44000A005573696E6720454550524F4D2073A7
:107A5400657474696E67730D0A005573696E6720E7
:107A640044656661756C742053657474696E6773DC
:107A74000D0A002D2D2D2D2D2D2D2D2D2D2D2D2DA2
:107A84002D2D2D2D2D2D2D2D2D2D2D2D2D2D2D2D22
:107A94002D2D2D2D2D2D2D2D2D2D2D2D2D2D2D2D12
:107AA4002D2D2D2D2D2D2D2D2D2D2D2D2D0D0A0072
:107AB4005374617274696E672050726F6365737377
:107AC4005061636B65740D0A004461746120696ED2
:107AD400206275666665723A200020627974657367
:107AE4000D0A004F564552464C4F572121210D0A8D
:107AF400004170706C79696E67206D6F64756C6F8E
:107B040020746F2072656164506F696E7465720DC4
:107B14000A004164647265737320666F72206C6539
:107B24006E3A0054465450205061636B6574205380
:107B3400697A653A004E6577205265616420506F1A
:107B4400696E7465723A006279746573746F7265F4
:107B540061643A005468697320697320626C6F63CE
:107B64006B206EB0004F70636F64653D00697320D5
:107B7400696E76616C6964206F70636F64650D0A69
:107B840000577269746520726571756573740D0AA6
:107B9400004368616E67656420746F20706F72744F
:107BA400200057726974696E6720446174612066AD
:107BB4006F7220626C6F636B206EB000466C6173F1
:107BC400682069732066756C6C210D0A0057726910
:107BD40074696E6720646174612066726F6D2061E0
:107BE4006464726573732000496E76616C69642005
:107BF400496D616765210D0A00466C6173682069EF
:107C04007320636F6D706C6574650D0A0041636B5E
:107C14000D0A004572726F720D0A0053656E64207E
:107C240041434B20284E6F742046696E616C290DC8
:107C34000A0053656E642041434B20005265737003
:107C44006F6E73652073656E740D0A00696D675FEE
:107C540073746174005446545020436F6D706C65A6
:107C640074650D0A00446F776E6C6F616420696EF1
:107C7400746572727570746564210D0A0052652D05
:107C8400696E697469616C6973696E6720544654DE
:107C940050207365727665722E2E2E0D0A0054697B
:0A7CA4006D656F7574210D0A000074
:040000030000700089
:00000001FF
